:020000040000FA
:020000000828CE
:020008000828C6
:1000100083123F30850000308600803087008C01DD
:10002000831606309F000F30850000308600983020
:100030008700403099002430980094171413093039
:100040009300FA30920083123030900027309500F0
:100050000C309700033092009030980028309400C4
:1000600007118512F001071487143F30B123C03007
:10007000B1235A21A901A801071487104930F200C1
:1000800032214830F20032214D30F200322120304E
:10009000F20032215630F20032216130F20032217A
:1000A0003630F2003221282404241A080A30C20013
:1000B000522331306B23642398181812181618191C
:1000C0001A088C1E6B281A08F200113A031D132916
:1000D00010100C1096280C1C5C2810100C106423B7
:1000E000C20B5C285528732C71187828851DBD2BF0
:1000F0000519872865306B23711010100C103124FE
:100100007012F1195A21F111282404248A288C1E16
:1001100073288F289818181218168C1E8A281A0807
:10012000F200313A031D162911306B237123720836
:10013000023A031D192971237208303A031D1E2942
:1001400071237208AB00803A031974297208403A8F
:10015000031DAD28F014F115C4287208483A031D98
:10016000B428F014F111C4287208F039AB002B0840
:10017000103A0319C4282B08203A0319C7282B0862
:10018000303A0319CA28212907148710CC280710F0
:100190008714CC2807148714A801A901720807390D
:1001A000A907A03084008312712372088000033AEB
:1001B0000319E7287208043A0319E6287208800038
:1001C000840A0408EF3A03190828D3287014F01C95
:1001D000F4282908AD005A212824F11D042407140D
:1001E0008710F0102D08A900A0308400A801000895
:1001F000F200033A031908297208043A031908297E
:1002000072083221840A0408EF3A03190828F728F3
:1002100070180D2906306B23A028071087100630B0
:100220006B23701073283030AF0024293130AF00B9
:1002300024293230AF0006306B2324293330AF003D
:1002400024293430AF00242907108714A9017D2305
:100250002E30A80081237208FE00C4242F08F2006B
:1002600032215528F30083120A3A03194C297D23C1
:1002700081238A1500208A112008AD232108AD238F
:100280002208AD232308AD232408AD230030AD237D
:100290002808063EA80008007D232808403A031DD0
:1002A0005529A801A90A7D23080081230030AD2328
:1002B000A80A4C2907148714A9017D23A8018123CA
:1002C0000030AD23A80A2808403A031D6029A90A76
:1002D0002908083A03196E297D235E290800A80120
:1002E0008123A9017D23080071237208B0007123C6
:1002F0007208B10071237208B20071237208B30052
:1003000071237208BB0071237208B8007123720850
:10031000B90071237208043A031D892970147114FD
:10032000F018F5295D235A21F014A901A80107143A
:1003300087100130A900A8012D30F200322133309E
:10034000F20032213030F200322136230230A9008F
:10035000A8012D30F20032213430F2003221303049
:10036000F200322136230330A900A8012D30F2001B
:1003700032213530F20032213030F2003221362382
:100380000430A900A8012D30F20032213630F200ED
:1003900032213030F200322136230530A900A80185
:1003A0002D30F20032213730F20032213030F200AD
:1003B000322136230630A900A8012D30F200322167
:1003C0003830F20032213030F2003221362307304B
:1003D000A900A8012D30F20032213930F20032217B
:1003E0003030F2003221362370113908003A031DF3
:1003F000FE29F0111830BA00C000092A3908273A3E
:10040000031D042AF011092A3908283A031D092A74
:10041000F015F01D172A0710871428303902BA008A
:100420008317A0303A0784000008C100222A07146D
:10043000871018303907BA00831720303907840035
:100440000008C10083133A0840060319372A701FB9
:100450002C2A071087142E2A071487104008A8009A
:100460003B08AE004108BB00CD222E08BB00F01DAA
:100470003D2A071087147017402A0714871070133D
:100480000130A9002908083A03194E2A7D233A08A9
:10049000C000A80081234523A90A422A0714871017
:1004A000A9017D23A80181233008F20032213108FF
:1004B000F20032213208F20032213308F2003221F8
:1004C0004D30F20032216830F20032217A30F200F1
:1004D000322107108714A9017D23A80181232D3023
:1004E000F2003221410889246430F2003221623066
:1004F000F20032216D30F20032213808003A031D3B
:10050000852A1830AC0070118B2A3808283A031D50
:100510008B2AAC017015701D992A0710871428309A
:100520003802AC008317A0302C0784003B08800001
:10053000A42A0714871018303807AC00831720301E
:10054000380784003B08800083132C08A800CD22C4
:1005500006306B2370100C1CC82A1010051CB42A1E
:10056000851CBE2AF013C82A8518BE2AF01BC82A8B
:100570002B306B230C105D23F0177429051CC82A3F
:10058000F01BC82A2D306B230C105D23F017742943
:10059000051D7A2811306B2374293B08633C03182E
:1005A000DC2A0130A90081237D234223A90A2908DE
:1005B000073A0319482BD32A0130A9001E303B0209
:1005C000A6000A30A602031CEA2A81237D234223C7
:1005D000A90AE12A0A30A60781237D232608003ACA
:1005E0000319162B2608013A0319192B2608023A7B
:1005F00003191C2B2608033A03191C2B2608043A5E
:1006000003191F2B2608053A0319222B2608063A40
:100610000319252B2608073A0319282B2608083A20
:100620000319282B2608093A03192B2BFF30AD2379
:100630002D2BFE30AD232D2BFC30AD232D2BF83090
:10064000AD232D2BF030AD232D2BE030AD232D2B02
:10065000C030AD232D2B8030AD23A90A2908083ADC
:10066000031908007D2381233F232D2B0130AD2367
:100670000130AD230130AD23FF30AD230800FF3042
:10068000AD2308000030AD2308005530AD2308002D
:1006900081237D238030AD230800E7308F00953023
:1006A0008E00562B0B308F00DB308E0031309000E7
:1006B0000C1C582B10100C100800EC308F007730F9
:1006C0008E003130900008000B308F00DB308E0040
:1006D00031309000080099008316981C6D2B83120E
:1006E00008008312181D752B1A089818181218166E
:1006F0008C1E782B1A08F20008002908B83EB12396
:1007000008002808403EB12308009B230516071463
:1007100087148316FF308600831287128516000027
:100720000000861B912B85128316003086008312F1
:100730000512A4230800071CF1100718F114871CE8
:100740007111871871150800F11C0710F1180714B2
:10075000711D8710711987140800A700852387165B
:10076000B42BA7008523871205122708860085165B
:100770000000000085128716080083123B244124E4
:1007800045244C2456245D242508FF3A0319732878
:10079000251CD92BA51CDF2B251DE12BA51DE32B2B
:1007A000251EE52BA51EEB2B251FF12BA51FFF23D7
:1007B0007328701ADD2B6330FA2B6F30FA2B2A3036
:1007C000FA2B5A30FA2B6230FA2B701AE92B3F3091
:1007D000FA2B4330F62B701AEF2B7330FA2B613063
:1007E000F62B701AF52B6D30FA2B4D30C3002824F0
:1007F000042443086B231215522312117328701E10
:10080000112C022C282431241030AD232030AD23AC
:100810007F30AD232030AD231030AD237012522332
:100820000800701628248316C830920083126430A2
:1008300095001215522312110430AD230230AD235E
:100840007F30AD230230AD230430AD2352230800A6
:10085000071487100730A9007D233630A8008123B4
:1008600008008316FA30920083127D30950012152D
:1008700052231211080063248316111483120313E8
:100880000800632441309300080063248316111B81
:10089000472C8312031308006324831691159119C2
:1008A0004F2C831203131308A5000800632483163A
:1008B0009116111683120313080063248316111571
:1008C0008312031308008316111A642C9119642CE7
:1008D0001119642C9118642C1118642C1419642CAF
:1008E000831203130800051C792C851C812CF0133E
:1008F00074288518812CF01B74282B306B23F0177B
:100900007328051C7328F01B74282D306B23F017F7
:1009100073280830AA00BD01BE01BF0105303D02A9
:100920000318B52405303E020318B82405303F02F1
:100930000318BB24AA030310C10DBF0D3F1ABE2428
:10094000BE0D3E1AC124BD0D03102A08031D8E2CB6
:100950003D08303EF20032213E08303EF2003221A6
:100960003F08303EF200322108000330BD07080086
:100970000330BE0708000330BF0708003F1203140E
:1009800008003E1203140800071087140730A9005E
:100990007D23A80181237E0E0F39FE1BE924303E02
:1009A000F20032217E080F39FE19E924303EF200B0
:1009B000322108007F0E0F39FF1BE924303EF20080
:1009C00032217F080F39FF19E924303EF20032212D
:1009D0000800AB00083A0319F42C2B08093A031954
:1009E000F62C2B08073E08000830080009300800E4
:101000007308F039303A031D32287308303A031957
:1010100058297308313A031963297308323A0319BE
:101020006E297308333A031979297308343A03197E
:1010300084297308353A03198F297308363A03193E
:101040009A297308373A0319A5297308383A0319FE
:10105000B0297308393A0319BB2973083E3A0319BA
:10106000C6294A297308F039403A031D74287308C9
:10107000413A0319D1297308423A0319DC2973084C
:10108000433A0319E7297308443A0319F22973080C
:10109000453A0319FD297308463A0319082A7308CB
:1010A000473A0319132A7308483A03191E2A73088A
:1010B000493A0319292A73084A3A0319342A73084A
:1010C0004B3A03193F2A73084C3A03194A2A73080A
:1010D0004D3A0319552A73084E3A0319602A7308CA
:1010E0004F3A03196B2A4A297308F039503A031D05
:1010F000A6287308503A0319762A7308513A03193F
:10110000812A7308523A03198C2A7308533A031937
:10111000972A7308543A0319A22A7308553A0319F7
:10112000AD2A7308563A0319B82A7308573A0319B7
:10113000C32A7308583A0319CE2A7308593A031977
:10114000D92A73085A3A0319E42A4A297308F0394C
:10115000603A031DE8287308613A0319EF2A7308FF
:10116000623A0319FA2A7308633A0319052B7308C4
:10117000643A0319102B7308653A03191B2B730883
:10118000663A0319262B7308673A0319312B730843
:10119000683A03193C2B7308693A0319472B730803
:1011A0006A3A0319522B73086B3A03195D2B7308C3
:1011B0006C3A0319682B73086D3A0319732B730883
:1011C0006E3A03197E2B73086F3A0319892B4A294B
:1011D0007308F039703A031D22297308703A031915
:1011E000942B7308713A03199F2B7308723A0319F1
:1011F000AA2B7308733A0319B52B7308743A0319B1
:10120000C02B7308753A0319CB2B7308763A031970
:10121000D62B7308773A0319E12B7308783A031930
:10122000EC2B7308793A0319F72B73087A3A0319F0
:10123000022C73087B3A0319392C73087D3A031981
:10124000442C4A2973081F3A0319702C73080C3A6E
:1012500003194B2973082C3A03190D2C73082D3AE6
:101260000319182C7308233A0319232C7308203A06
:1012700003192E2C73080D3A031954297308283AC0
:1012800003194F2C73082E3A03195A2C73082F3A5E
:101290000319652C0800A001A101A201A301A4016A
:1012A0008A115A218A1508008A116F218A150800AF
:1012B0003E30A0005130A1004930A2004530A300CB
:1012C0007E30A4004A290030A0004230A1007F30C7
:1012D000A2004030A3000030A4004A294230A00000
:1012E0006130A1005130A2004930A3004630A40073
:1012F0004A292130A0004130A1004530A2004B30E6
:10130000A3003130A4004A291830A0001430A100F5
:101310001230A2007F30A3001030A4004A292730E9
:10132000A0004530A1004530A2004530A30079302F
:10133000A4004A297C30A0004A30A1004930A20014
:101340004930A3003030A4004A290130A000713098
:10135000A1000930A2000530A3000330A4004A29EF
:101360003630A0004930A1004930A2004930A30026
:101370003630A4004A290630A0004930A100493087
:10138000A2002930A3001E30A4004A290030A0008A
:101390004130A1002230A2001430A3000830A40084
:1013A0004A297E30A0000930A1000930A20009308E
:1013B000A3007E30A4004A297F30A0004930A1005C
:1013C0004930A2004930A3003630A4004A293E30FB
:1013D000A0004130A1004130A2004130A3002230E2
:1013E000A4004A297F30A0004130A1004130A20072
:1013F0002230A3001C30A4004A297F30A0004930CD
:10140000A1004930A2004930A3004130A4004A297C
:101410007F30A0000930A1000930A2000930A300EC
:101420000130A4004A293E30A0004130A1004930DB
:10143000A2004930A3007A30A4004A297F30A000DE
:101440000830A1000830A2000830A3007F30A400BB
:101450004A290030A0004130A1007F30A200413075
:10146000A3000030A4004A292030A0004030A10091
:101470004130A2003F30A3000130A4004A297F3050
:10148000A0000830A1001430A2002230A300413097
:10149000A4004A297F30A0004030A1004030A200C3
:1014A0004030A3004030A4004A297F30A000023021
:1014B000A1000C30A2000230A3007F30A4004A2912
:1014C0007F30A0000430A1000830A2001030A3003B
:1014D0007F30A4004A293E30A0004130A1004130B5
:1014E000A2004130A3003E30A4004A297F30A00072
:1014F0000930A1000930A2000930A3000630A40081
:101500004A293E30A0004130A1005130A2002130D4
:10151000A3007E30A4004A297F30A0000930A1003A
:101520001930A2002930A3004630A4004A294630D1
:10153000A0004930A1004930A2004930A300313059
:10154000A4004A290130A0000130A1007F30A20090
:101550000130A3000130A4004A293F30A0004030F0
:10156000A1004030A2004030A3003F30A4004A292F
:101570001F30A0002030A1004030A2002030A30086
:101580001F30A4004A293F30A0004030A1003F3066
:10159000A2004030A3003F30A4004A296330A000DD
:1015A0001430A1000830A2001430A3006330A4005E
:1015B0004A290730A0000830A1007030A20008308E
:1015C000A3000730A4004A296130A0005130A100D7
:1015D0004930A2004530A3004330A4004A292030FE
:1015E000A0005430A1005430A2005430A300783041
:1015F000A4004A297F30A0004830A1004430A20056
:101600004430A3003830A4004A293030A0004830CC
:10161000A1004830A2004830A3002030A4004A298D
:101620003830A0004430A1004430A2004830A3006C
:101630007F30A4004A297830A0005430A1005430F3
:10164000A2005430A3001830A4004A290830A0009A
:101650007E30A1000930A2000130A3000230A400B6
:101660004A290C30A0005230A1005230A200523062
:10167000A3003E30A4004A297F30A0000830A1001A
:101680000430A2000430A3007830A4004A290030BE
:10169000A0004430A1007D30A2004030A300003003
:1016A000A4004A292030A0004030A1004430A2000C
:1016B0003D30A3000030A4004A297F30A000103044
:1016C000A1002830A2004430A3000030A4004A2921
:1016D0000030A0004130A1007F30A2004030A300C4
:1016E0000030A4004A297C30A0000430A10018304A
:1016F000A2000430A3007830A4004A297C30A00066
:101700000830A1000430A2000430A3007830A40007
:101710004A293830A0004430A1004430A2004430AF
:10172000A3003830A4004A297C30A0001430A10066
:101730001430A2001430A3000830A4004A29083055
:10174000A0001430A1001430A2001830A3007C3097
:10175000A4004A297C30A0000830A1000430A20077
:101760000430A3000830A4004A294830A0005430B7
:10177000A1005430A2005430A3002030A4004A2914
:101780000430A0003F30A1004430A2004030A3004C
:101790002030A4004A293C30A0004030A100403055
:1017A000A2002030A3007C30A4004A291C30A000F5
:1017B0002030A1004030A2002030A3001C30A40043
:1017C0004A293C30A0004030A1003C30A20040300B
:1017D000A3003C30A4004A294430A0002830A100D6
:1017E0001030A2002830A3004430A4004A294C3015
:1017F000A0005030A1005030A2005030A3003C3077
:10180000A4004A294430A0006430A1005430A20052
:101810004C30A3004430A4004A290030A0005030CE
:10182000A1006030A2000030A3000030A4004A29CB
:101830000030A0000830A1000830A2000830A3004A
:101840000030A4004A291430A0007F30A1001430D9
:10185000A2007F30A3001430A4004A290030A00069
:101860000030A1000030A2000030A3000030A4002E
:101870004A298030A000F630A100E630A200D63020
:10188000A300B930A4004A29FE30A000FE30A10018
:101890008030A200FE30A300FE30A4004A29803030
:1018A000A000FD30A100F330A200FD30A300803085
:1018B000A4004A290030A0006030A1006030A200DE
:1018C0000030A3000030A4004A292030A0001030CE
:1018D000A1000830A2000430A3000230A4004A296D
:1018E0000030A0000030A1000F30A2000930A3009A
:0618F0000F30A4004A299C
:02400E00723FFF
:00000001FF
